:0A0000000C948B030C9400000C9488
:10000A0000000C9400000C9400000C94AD150C94A4
:10001A0000000C9495150C9400000C9400000C94AC
:10002A0000000C9400000C94DA150C9400000C9457
:10003A0000000C9400000C9400000C9400000C9436
:10004A0043150C9400000C9400000C9400000C94CE
:10005A0000000C9400000C9400000C9400000C9416
:10006A0000000C9400000C9400000C9400000C9406
:10007A0000000C9400000C9400000C9400000C94F6
:10008A0000001027E80364000A00010000100001C4
:10009A0010000100140048005D0078009600B600C8
:1000AA00D500F30010012C01490163017C01940180
:1000BA00AC01C101D501E801543D2025750A47006C
:1000CA00533D2025750A53004E3D2025750A5700D9
:1000DA004B3D2025750A5600503D332E340A5200F6
:1000EA004C3D2025750A68004F3D73740A5300473A
:1000FA003D73740A5300523DD1F2E0EDF6E8FF0A6F
:10010A005700523DC2C5D0D50A5700523DCFEEE442
:10011A00EEE3F0E5E20A5700523DD0E5E1EEEBEB03
:10012A00E8EDE30A5700523DD0F3F7EDEEE90A573E
:10013A0000503D536E36332F506233370A57005002
:10014A003D536E41670A5700503DCFF0EEF4E8EB9D
:10015A00FC20300A5700503DCFF0EEF4E8EBFC20CB
:10016A00310A5700503DCFF0EEF4E8EBFC20320A9A
:10017A005700503DCFF0EEF4E8EBFC20330A57006D
:10018A00503DCFF0EEF4E8EBFC20340A5700503D26
:10019A00CFF0EEF4E8EBFC20350A5700503DCDE5F0
:1001AA00F20A5700D1D2C0CDD6C8DF202000C2C57E
:1001BA00D0D5202020202000CFCEC4CEC3D0C5C2A7
:1001CA002000D0C5C1CECBCBC8CDC3002020202073
:1001DA00D0D3D7CDCEC920D0C5C6C8CC20202020A8
:1001EA0000D1D2C5CACBCE00C4EEEF2E20CDE0F1AD
:1001FA00F2F0EEE9EAE80020536E36332F5062330C
:10020A003700202020202020536E416700CFD0CE17
:10021A00D4C8CBDC203000CFD0CED4C8CBDC203140
:10022A0000CFD0CED4C8CBDC203200CFD0CED4C8B9
:10023A00CBDC203300CFD0CED4C8CBDC203400CFE7
:10024A00D0CED4C8CBDC20350048C8C72020202A0D
:10025A00D1D2C0D0D22A202020424550580048C8C6
:10026A00C7202020202AD1D2CECF2A2020204245C2
:10027A005058005057253375202A2534752A2020D6
:10028A0050572533750074253375B04320742533D0
:10029A0075B0432074253375B043002020202020F8
:1002AA002020202020202020202020202020200064
:1002BA00C2FBE1EEF020F0E5E6E8ECE020F1F2E046
:1002CA00EDF6E8E800C2FBE1EEF020EFF0EEF4E82C
:1002DA00EBFF20EFE0E9EAE8200020202054552B2C
:1002EA00253475B043202020002020202054454D7D
:1002FA005025337520202020202020200020202077
:10030A002020204B3D25327520202020202020202F
:10031A000020202020202AC2CACBDED7C5CD2A2021
:10032A0020202020200020202020202AC2DBCACB27
:10033A00DED7C5CD2A202020202000202020202002
:10034A0020253475B04320202020202000202020A2
:10035A002020202020253375202020202020202026
:10036A00002ACDC0D1D2D0CEC9CAC02020CFD0CE8B
:10037A00D4C8CBDF2A0020202020D2C5CCCFC5D0BC
:10038A00C0D2D3D0C020202020200020202020CC82
:10039A00C5D1D2C020CFC0C9CAC820202020200081
:1003AA00CDC8C6CDC5C3CE20CDC0C3D0C5C2C0D26C
:1003BA00C5CBDF002020D2C5CCCFC5D0C0D2D3D088
:1003CA00C020C2CACB2E202000C2C5D0D5CDC5C3FD
:1003DA00CE20CDC0C3D0C5C2C0D2C5CBDF0020203D
:1003EA00202020CA2DCFD0CED4C8CBDF2020202079
:1003FA00202000CDC8C6CDC5C3CE2020CDC0C3D0D5
:10040A00C5C2C0D2C5CBDF00202020D0C5C6C8CC0B
:10041A0020CACECDD2D0CECBDF2020200020D4D30C
:10042A00CDCAD6C8DF20C4CECDC0C3D0C5C2C02075
:10043A0020002020202020C4CECDC0C3D0C5C2C0F9
:10044A0020202020202000202020D2C5CCCF2EC45E
:10045A00CECDC0C3D0C5C2C020202000202020207D
:10046A004D415820CCCED9CDCED1D2DC202020206F
:10047A0000202020204D415820CCCED9CDCED1D23B
:10048A00DC202020002020C4CED1D2C8C6C5CDC8C9
:10049A00DF20D2C5CCCF2E202000202020CDC0C303
:1004AA00D0C5C2C020CFCBC0D2DB20202020002064
:1004BA002020202020CDC8C72BC2C5D0D52020207F
:1004CA00202020002020202020D2CECBDCCACE2023
:1004DA00CDC8C720202020200020202020D2CECB2B
:1004EA00DCCACE2020C2C5D0D52020202000202062
:1004FA0020202020CED2CACBDED7C5CD2020202076
:10050A0020200020202025347520F1E5EA20202033
:10051A000020202020202020D0C5C6C8CC202020A2
:10052A002020202020002020202020D0C5C1CECB92
:10053A00CBC8CDC3C020202020200020C2C5D0D5E2
:10054A002E20CDC0C3D0C5C2C0D2C5CBDF2020006B
:10055A0020202020202020C2D0C5CCDF202020202F
:10056A002020202000202020C4CECFCECBCDC8D240
:10057A00C5CBDCCDDBC5202020002020202020CDCB
:10058A00C0D1D2D0CEC9CAC8202020202020002025
:10059A0020202020E2E5F0F1E8FF20342E30202050
:1005AA00202020002020202020202AC2DBD5CEC4F3
:1005BA002A2020202020202000202AC4C0D2D7C8E8
:1005CA00CA20312028C2C5D0D5292A2020002020BF
:1005DA002020205455253375202020202020002A51
:1005EA00C4C0D2D7C8CA20322028CDC8C6CDC8C9EF
:1005FA00292A200020202020205444253375202039
:10060A0020202020002020202AC2D0C5CCDF20CFE5
:10061A00C0C9CAC82A20202020002020202020204B
:10062A00205455253375202020202020202000200A
:10063A002020CFD0C5C420D3D1D2C0CDCEC2CAC803
:10064A00202020002020202020D3D1D2C0CDCEC20D
:10065A00CBC5CDDB202020202000202020202020F8
:10066A0020202020202020202020202020202000A0
:10067A00202055534220CFCEC4CACBDED7C5CDC821
:10068A00C520202000202020202ACFCEC4CACBDEBD
:10069A00D7C5CDCE2A202020200020202ACDC52053
:1006AA00CFCEC4CACBDED7C5CDCE2A20202000208B
:1006BA0020202020202020C7C2D3CA20202020208A
:1006CA0020202000202020202020C2DBCACBDED719
:1006DA00C5CD20202020202000202020202020C23C
:1006EA00CACBDED7C5CD202020202020200080C004
:1006FA0001002D4E414E000024006D059E000200AF
:10070A00C705F8060100CE05FA060000F894EE27A0
:10071A00ECBBF1E0F5BFE5BFE0936C00F8E1F1BD99
:10072A00E1BD8DE0A2E0BB27ED938A95E9F780E071
:10073A0090E1A0E0B1E0ED930197E9F7E2E0F7E09C
:10074A0085919591009761F0A591B59105901590C5
:10075A00BF01F00105900D920197E1F7FB01F0CF7F
:10076A00EFEFEDBFE0E1EEBFC0E0D5E00C941A1662
:10077A001A930A93B89AC09A0E943C1AC0980E9487
:10078A00441AE0936505F093660589E18A95F1F7C5
:10079A000E94441AE0936905F0936A05C09AE091B1
:1007AA006505F09166050E944A1ADF01CB01E091C6
:1007BA006905F0916A050E94521AA1EAB1E027C0C0
:1007CA001A930A93A79AAF9A0E943C1AAF980E946A
:1007DA00441AE0936705F093680589E18A95F1F771
:1007EA000E94441AE0936B05F0936C05AF9AE0916E
:1007FA006705F09168050E944A1ADF01CB01E09172
:10080A006B05F0916C050E94521AA3EAB1E00E94AE
:10081A00541F0E94FD1E0E94E31FDF01CB01E0E08E
:10082A00F0E068EC72E40E94B220ADECBCEC8CEC17
:10083A009DE30E941620D801882799270E94441F09
:10084A000E9464200E94AA1F8F01F8010991199140
:10085A000895A895B5DFE0933C05F0933D050E9405
:10086A00601AA935E2E0BE0730F0E7EEF3E0E09364
:10087A003C05F0933D050E94651A7ADFE0933E0538
:10088A00F0933F050E946B1AA935E2E0BE0730F0EB
:10089A00E7EEF3E0E0933E05F0933F05A89508954F
:1008AA000E94701A59F4E1E0E51541F4A09140055F
:1008BA00A33521F43ED1E0E0E09340050E94701A8E
:1008CA0069F4552059F4A0914005AA3519F4E1E0DC
:1008DA00E0934105A0914105A130E1F3E2ECF0E09B
:1008EA000E94761A0E947D1AEAECF0E0FA93EA93E3
:1008FA00E0913605F09137050E947D1AE2EDF0E0AD
:10090A00FA93EA930E94861A0E948B1AEAEDF0E0A3
:10091A00FA93EA930E94941A0E948B1AE2EEF0E08C
:10092A000E94991AEAEEF0E0FA93EA930E94A01A5A
:10093A000E947D1AE1E0E51521F4E2EFF0E00E9461
:10094A00991A552021F4E9EFF0E00E94991A0E94C1
:10095A00A51A19F4E0E0F1E01BC0E130A0E0FA07C3
:10096A0019F4ECE0F1E014C0E230A0E0FA0719F45F
:10097A00E5E1F1E00DC0E330A0E0FA0719F4E2E2A4
:10098A00F1E006C0E430A0E0FA0741F4E0E3F1E068
:10099A00FA93EA9380E00E940D1A2296442011F0FD
:1009AA000C941805E72D0E94A91A19F40E94AC1A92
:1009BA003AC0E130A0E0FA0719F40E94AF1A33C036
:1009CA00E230A0E0FA0719F40E94B21A2CC0E33010
:1009DA00A0E0FA0729F4E0E6F1E00E94991A23C0A0
:1009EA00E430A0E0FA0729F4EEE6F1E00E94991A51
:1009FA001AC0E530A0E0FA0729F4ECE7F1E00E941A
:100A0A00991A11C0E630A0E0FA0729F4EAE8F1E001
:100A1A000E94991A08C0E730A0E0FA0721F4E8E931
:100A2A00F1E00E94991AE1E0E415A1F4EA2D0E948E
:100A3A00A91A19F40E94AC1A0DC0E130A0E0FA0715
:100A4A0019F40E94AF1A06C0E230A0E0FA0711F4C6
:100A5A000E94B21AE2E0E415A1F4EB2D0E94A91A51
:100A6A0019F40E94AC1A0DC0E130A0E0FA0719F49B
:100A7A000E94AF1A06C0E230A0E0FA0711F40E9401
:100A8A00B21AE3E0E41531F5ED2D0E94A91A19F422
:100A9A000E94AC1A1FC0E130A0E0FA0719F40E94C4
:100AAA00AF1A18C0E230A0E0FA0719F40E94B21A8D
:100ABA0011C0E330A0E0FA0729F4E0E6F1E00E9471
:100ACA00991A08C0E430A0E0FA0721F4EEE6F1E052
:100ADA000E94991AE4E0E41521F4E6EAF1E00E94A2
:100AEA00991A0895AC9AA8950AC0AC9AA8950E943A
:100AFA00B51AAC98A8950E94B51AAC9AA8950E9406
:100B0A00B51AAC980895AC9A0E94B51AAC98A895F3
:100B1A000E94B51AAC9AA8950E94B51AAC98A895E5
:100B2A000E94B51AAC9AA8950E94B51AAC98A895D5
:100B3A0008950E94BB1A5524E6DF0895A0E0B0E0AC
:100B4A00E3ECF0E00E94641FA2E0B0E00E94D01A39
:100B5A00A4E0B0E0EEE6F0E00E94641FA6E0B0E098
:100B6A000E94D51AA8E0B0E00E94D51AAAE0B0E027
:100B7A000E94DA1AACE0B0E0E1E0F0E00E94641F03
:100B8A00AEE0B0E00E94DA1AA0E1B0E00E94DA1A00
:100B9A00A2E1B0E00E94DF1AA4E1B0E00E94DF1AED
:100BAA00A8E1B0E0E6EEF0E00E94641FAAE1B0E03E
:100BBA000E94D01AACE1B0E0E3E7F0E00E94641FC3
:100BCA00AEE1B0E00E94D51AA0E2B0E00E94D51AC8
:100BDA00A2E2B0E00E94DA1AA4E2B0E0E1E0F0E0BA
:100BEA000E94641FA6E2B0E00E94DA1AA8E2B0E00E
:100BFA000E94DA1AAAE2B0E00E94DF1AACE2B0E080
:100C0A000E94DF1AA0E3B0E0E6EEF0E00E94641F63
:100C1A00A2E3B0E00E94D01AA4E3B0E0E9E6F0E073
:100C2A000E94641FA6E3B0E00E94D51AA8E3B0E0D0
:100C3A000E94D51AAAE3B0E00E94DA1AACE3B0E047
:100C4A000E94DA1AAEE3B0E0E2EDF0E00E94641F1F
:100C5A00A0E4B0E0E9E1F0E00E94641FA2E4B0E0A1
:100C6A000E94DF1AA4E4B0E00E94DF1AAAE0B1E011
:100C7A00E0E9F1E00E94641FACE0B1E0E2E8F0E0F4
:100C8A000E94641FA0E1B1E0E8E1F0E00E94641F65
:100C9A00A2E1B1E00E94DA1AA0ECB0E0ECEDF0E0DB
:100CAA000E94641FA4ECB0E0EEE6F0E00E94641F2C
:100CBA00A6ECB0E0E4E1F0E00E94641FAAECB0E028
:100CCA000E94DA1AA4EDB0E00E94DF1AA2E5B1E0B0
:100CDA00ECE2F1E00E94641FAAE5B1E00E94DA1A90
:100CEA00A4E6B1E0EAE5F0E00E94641FAEE5B1E0F7
:100CFA00E4EAF1E00E94641FA1EAB1E0EFE0F0E06B
:100D0A000E94641FA3EAB1E00E94641FA7EAB1E04F
:100D1A00EAE0F0E00E94641F55240E94E41AA8E960
:100D2A00B1E0E0E00E946C1F4424E0E0F0E00E94A1
:100D3A00EB1AE0E0F0E0E0933005F09331050E9411
:100D4A00F01AA9E9B1E00E94DA1AABE9B1E00E940F
:100D5A00DA1AADE9B1E00E94DA1AAFE9B1E00E940D
:100D6A00DA1AA6EAB1E0E1E00E946C1FA5EAB1E056
:100D7A000E946C1FE4E0E0935D050895A895E0E009
:100D8A00E0936105E0936005E0936205CC240E943C
:100D9A00F71A0E94FE1A0E94051B0E940C1B089556
:100DAA000E94F9200E94131B0D911C910E941D1B89
:100DBA003196E09391050E94131B2D913C91AC81D1
:100DCA00BD810A171B07F8F4A895AC81BD81A2174B
:100DDA00B30770F40E941D1BA5E0B0E00E940F1F2C
:100DEA0032970E94211B0E941D1B3197E0939105A7
:100DFA00EC81FD810E94261BEA17FB0720F4E4E13F
:100E0A00F0E00E94211BA8950E942B1B0E94301B18
:100E1A00EA17FB0710F40E94351BA8950E940021CF
:100E2A0026960895E0916105E03011F00C942A08A5
:100E3A00E0916205E03051F40E94371B10F40E94E1
:100E4A003C1B0E943F1B10F00E94441B0E94471B40
:100E5A0014F40E945A1B0E945D1B14F00E943C1B52
:100E6A00A895A0916205A13091F5E0916005E03066
:100E7A0021F50E94621BAE17BF07F8F40E946B1B94
:100E8A0068F40E94731B0E94781B10F40E94351BA1
:100E9A000E945D1B14F00E943C1B0FC00E94301B75
:100EAA0011972CF00E94731B3197FE93EE930E94C8
:100EBA00301B119714F40E945A1B0E94801B3A9708
:100ECA000E94851B20F4E6E4F0E00E94211BA8950D
:100EDA000E94891BA1F4E0916005E03081F40E9430
:100EEA008F1B68F00E94941BE2E3F0E00E94211B32
:100EFA00E1E0E0935005F6DDE1E0E0936005A091C2
:100F0A006005A13011F40E949C1B0E94621BEA1723
:100F1A00FB0728F40E94A41B11F40E94AA1B0E943A
:100F2A00B41B0E94B91B0E94BE1B14F40E94CF1B63
:100F3A00A8950E94D61B0E94DB1B10F40E94E21B9C
:100F4A000E94E81B0E94ED1BEA17FB0710F40E949F
:100F5A00F21BA8950E94801B0E94851BE8F40E9440
:100F6A00F81B58F40E94FD1B38F40E94051C0E94CD
:100F7A000A1C14F00E94121C0FC00E94ED1B11974C
:100F8A002CF00E94051C3197FE93EE930E94ED1BF4
:100F9A00119714F40E94CF1B0E94D61B0E94851B36
:100FAA0098F50E94ED1B11972CF00E94051C3197B1
:100FBA00FE93EE930E94191C369760F00E94ED1B77
:100FCA001A9714F40E94CF1B0E94ED1B1A9714F073
:100FDA000E94241CE0916105E03039F40E947A05F0
:100FEA00E1E0E0935205E09361050E942B1C0E9408
:100FFA00301C50F4E1E0E09361050E94CF1B0E948F
:10100A005A1B81DDE1E05E2EA8950E94371CE1F4AF
:10101A00CC20D1F40E943D1CE0913E05F0913F05A1
:10102A00EA1BFB0B359780F40E94421CA0916305D2
:10103A00B0916405EA0FFB1FE0936305F093640522
:10104A000E947705E1E0CE2EA8950895A895E09133
:10105A006105E03011F00C94B508E0916005E030CC
:10106A0039F50E94B41BA0913605B09137050E944C
:10107A00BE1B14F40E94CF1BA8950E94D61B0E9487
:10108A00DB1B10F40E94E21B0E94191C329780F4A9
:10109A00E2E3F0E0E0934805F0934905E1E0E093EC
:1010AA006005E09350050E94A41B11F40E947A0582
:1010BA00A8950E94E81B0E94ED1BEA17FB0710F493
:1010CA000E94F21BA8950E94F81BD0F40E94FD1BF7
:1010DA0040F40E94051C0E940A1C14F00E94121C73
:1010EA000FC00E94ED1B11972CF00E94051C31972E
:1010FA00FE93EE930E94ED1B119714F40E94CF1BEE
:10110A00A8950E94D61B0E94851BC8F40E94ED1B5D
:10111A0011972CF00E94051C3197FE93EE930E94C2
:10112A00191C369760F00E94ED1B1A9714F40E945E
:10113A00CF1B0E94ED1B1A9714F00E94241CA8953D
:10114A000E94B91BAD32E1E0BE0750F0E0E0E09347
:10115A006005E1E0E09361050E94CF1B0E948805CB
:10116A00A8950895E0916105E03011F00C943209D8
:10117A00E0916205E03069F40E94371B10F40E9486
:10118A003C1B0E943F1B28F00E94441BE1E0E093B5
:10119A0062050E94891B71F4E0916005E03051F408
:1011AA000E948F1B38F00E94941B0E947705E1E091
:1011BA00E09360050E94471B14F40E945A1B0E9488
:1011CA005D1B14F00E943C1BA895A0916205A130FA
:1011DA0091F5E0916005E03021F50E94621BAE179F
:1011EA00BF07F8F40E946B1B68F40E94731B0E94ED
:1011FA00781B10F40E94351B0E945D1B14F00E949C
:10120A003C1B0FC00E94301B11972CF00E94731BCD
:10121A003197FE93EE930E94301B119714F40E94AB
:10122A005A1B0E94801B3A970E94851B20F4E6E411
:10123A00F0E00E94211BA895A0916005A13011F44D
:10124A000E949C1B0E94621BEA17FB0728F40E945B
:10125A00A41B11F40E94AA1BA8950895E0916105A8
:10126A00E03011F00C94C8090E94471C88F4E09100
:10127A006205E03069F40E94371B10F40E943C1B9F
:10128A000E943F1B28F0E1E0E09362050E94441BA4
:10129A000E94471CE1F4E1E0E0935005E09160050B
:1012AA00E030A9F40E94B91BA436E0E0BE0710F4AE
:1012BA000E94121C0E94B91BA536E0E0BE0738F056
:1012CA000E94F21BE1E0E0935105E09360050E9461
:1012DA00471C68F4A0916205A13049F40E944D1C94
:1012EA00FA93EA930E94D506E1E0E09350050E9442
:1012FA00A41BE1F4E0916005E03059F40E94B91BA7
:10130A00A536E0E0BE0728F00E94121CE1E0E09357
:10131A005105A0915505B0915605DD9738F00E9408
:10132A00F21BE1E0E0935205E09360050E94A41BE2
:10133A0051F40E94521C0E94301C28F40E94CF1BB8
:10134A00E1E0E09361050E94891B61F40E94521C4E
:10135A000E94B91BEA17FB0728F40E945A1BE1E016
:10136A00E09361050E94471C71F40E94521CA091EF
:10137A005505B0915605EA17FB0728F40E94CF1BC2
:10138A00E1E0E0936105A8950895E0E5F0E00E94A8
:10139A00571C0E946B1AAB35E0E0BE0710F00E94A2
:1013AA005A1BE0916205E03099F40E94601AA83C49
:1013BA00E0E0BE0710F40E943C1B0E94601AA93CA0
:1013CA00E0E0BE0728F00E947705E1E0E0936205BD
:1013DA00A0916205A13081F40E94601AA13AE0E06E
:1013EA00BE0710F00E945A1B0E94601AA837E0E05C
:1013FA00BE0710F40E94441BA8950895E8810E9434
:10140A00A91A39F40E945C1CEEEAF1E00E94611C00
:10141A0041C0E130A0E0FA0739F40E945C1CE8EB15
:10142A00F1E00E94611C36C0E230A0E0FA0739F40C
:10143A000E945C1CE2ECF1E00E94611C2BC0E330CC
:10144A00A0E0FA0739F40E945C1CECECF1E00E947F
:10145A00611C20C0E430A0E0FA0739F40E945C1C49
:10146A00E6EDF1E00E94611C15C0E530A0E0FA0744
:10147A0039F40E945C1CEBEEF1E00E94611C0AC088
:10148A00E630A0E0FA0731F40E945C1CE2EFF1E0DA
:10149A000E94611CD8C0E881E03011F00C94AC0ABB
:1014AA00E72D0E94A91A39F40E94651CE1E0F2E0D6
:1014BA000E94611C4CC0E130A0E0FA0739F40E9496
:1014CA00651CECE0F2E00E94611C41C0E230A0E041
:1014DA00FA0739F40E94651CE7E1F2E00E94611CF8
:1014EA0036C0E330A0E0FA0739F40E94651CE1E255
:1014FA00F2E00E94611C2BC0E430A0E0FA0739F444
:10150A000E94651CEBE2F2E00E94611C20C0E530FB
:10151A00A0E0FA0739F40E94651CE5E3F2E00E94B4
:10152A00611C15C0E630A0E0FA0739F40E94651C78
:10153A00EFE3F2E00E94611C0AC0E730A0E0FA077C
:10154A0031F40E94651CE9E4F2E00E94611CA88162
:10155A00A130F1F4EA2D0E94A91A29F40E94651C0F
:10156A00E1E0F2E011C0E130A0E0FA0729F40E94BC
:10157A00651CECE0F2E008C0E230A0E0FA0741F4B2
:10158A000E94651CE7E1F2E0FA93EA930E94BB1716
:10159A00A881A230F1F4EB2D0E94A91A29F40E9425
:1015AA00651CE1E0F2E011C0E130A0E0FA0729F49D
:1015BA000E94651CEEE0F2E008C0E230A0E0FA0703
:1015CA0041F40E94651CE7E1F2E0FA93EA930E9473
:1015DA00BB17A881A33021F5E2E0ED1508F4DD245C
:1015EA00ED2D0E94A91A39F40E94651CE7E1F2E088
:1015FA000E94611C15C0E130A0E0FA0739F40E948C
:10160A00651CE1E2F2E00E94611C0AC0E230A0E03F
:10161A00FA0731F40E94651CEBE2F2E00E94611CB9
:10162A0012C0E881E03031F40E946B1CE3E5F2E07D
:10163A000E94611CA881A13031F40E946B1CE8E66B
:10164A00F2E00E94611C219608950E94711CEDE748
:10165A00F2E0FA93EA93ED81FF27662777270E9443
:10166A003D1FE0913605F09137050E94761CEC8506
:10167A00FF27662777270E943D1F0E947B1C0E9436
:10168A00821C0E94711C0E94AE170E94B51AA8956E
:10169A000E94711CE0E9F2E0FA93EA93E885F98581
:1016AA000E94761C0E94861CEE85FF850E94761C8D
:1016BA000E947B1C0E94881C0E94711C0E94AE170B
:1016CA00A89526960895E0915A05E03009F4552424
:1016DA00A0915A05A13011F4E1E05E2E0895A0917F
:1016EA005B05A73039F40E94BB1A0E947705E1E036
:1016FA00E0935B05A0915B05A23039F40E94BB1A06
:10170A000E948805E1E0E0935B05E0915B05E0302B
:10171A0039F40E949A0C0E947705E1E0E0935B0598
:10172A0008954A926BDE999937C0A42D0E948C1CA9
:10173A004E2E0E94931C0E94961C0E946B1C0E94B3
:10174A00961C989B26C00E94991C58DE0E949E1CDB
:10175A00EAEBF2E00E94611CA895999905C04394AE
:10176A000E94A11C0E94961C999902C0A895FCCFC0
:10177A009A9905C04A940E94A11C0E94961C9A99A3
:10178A0002C0A895FCCFA895E6E0E41508F4442425
:10179A00D8CFE7E0E093590508954A927CDE9B99F9
:1017AA00C3C0A72D0E948C1C7E2EAA2D0E948C1CC1
:1017BA00AE2EAB2D0E948C1CBE2EAD2D0E948C1C11
:1017CA00DE2E0E94931C0E94961C0E946B1C0E9493
:1017DA00961C442041F5989B23C00E94991C0E94A4
:1017EA00A81C0E94AB1CA8959B9905C073940E94E3
:1017FA00A11C0E94961C9B9902C0A895FCCFCF9968
:10180A0005C07A940E94A11C0E94961CCF9902C01E
:10181A00A895FCCFA895E7E0E71508F47724DBCF75
:10182A00E7E0E0935905E1E0E41541F5989B23C010
:10183A000E94991C0E94A81C0E94AB1CA8959B9907
:10184A0005C0A3940E94A11C0E94961C9B9902C0E9
:10185A00A895FCCFCF9905C0AA940E94A11C0E940A
:10186A00961CCF9902C0A895FCCFA895E2E0EA158C
:10187A0008F4AA24DBCFE7E0E0935905E2E0E41597
:10188A0041F5989B23C00E94991C0E94A81C0E94A3
:10189A00AB1CA8959B9905C0B3940E94A11C0E94F9
:1018AA00961C9B9902C0A895FCCFCF9905C0BA9403
:1018BA000E94A11C0E94961CCF9902C0A895FCCF39
:1018CA00A895E2E0EB1508F4BB24DBCFE7E0E09350
:1018DA005905E3E0E41541F5989B23C00E94991C41
:1018EA000E94A81C0E94AB1CA8959B9905C0D39482
:1018FA000E94A11C0E94961C9B9902C0A895FCCF2D
:10190A00CF9905C0DA940E94A11C0E94961CCF9917
:10191A0002C0A895FCCFA895E2E0ED1508F4DD24F5
:10192A00DBCFE7E0E093590508951A930A930E94E2
:10193A00A51A81F400E010E00C30E0E01E074CF438
:10194A000E94AE1C0E94B71C0E94C21C0F5F1F4F50
:10195A00F3CF3BC0E130A0E0FA0781F400E010E0E9
:10196A000C30E0E01E074CF40E94AE1C0E94CA1C18
:10197A000E94C21C0F5F1F4FF3CF27C0E230A0E0C6
:10198A00FA0781F400E010E00C30E0E01E074CF4A6
:10199A000E94AE1C0E94D51C0E94C21C0F5F1F4FE2
:1019AA00F3CF13C0E330A0E0FA0779F400E010E0C7
:1019BA000C30E0E01E074CF40E94AE1C0E94E01CB2
:1019CA000E94C21C0F5F1F4FF3CFE0911005F091E8
:1019DA0011050E94571CE0911205F09113050E940F
:1019EA00EB1CE0911405F09115050E94F01CE091A2
:1019FA001605F09117050E94F51CE0911805F09163
:101A0A0019050E94FA1CE0911A05F0911B050E9423
:101A1A00FF1CE0911C05F0911D05E0932805F09349
:101A2A002905E0911E05F0911F050E94041DE09111
:101A3A002005F0912105E0932C05F0932D05E09106
:101A4A002205F09123050E94091DE0912405F091D9
:101A5A0025050E940E1D0E94C3068CC01A930A9384
:101A6A000E94D61BE0931005F09311050E944D1CAD
:101A7A00E0931205F09313050E94801BE09314056E
:101A8A00F09315050E94B41BE0931605F093170511
:101A9A000E94131DE0931805F0931905E091420581
:101AAA00F0914305E0931A05F0931B050E94181D57
:101ABA00E0931C05F0931D050E94521CE0931E053D
:101ACA00F0931F050E94421CE0932005F093210524
:101ADA000E942B1BE0932205F09323050E94E81B2A
:101AEA00E0932405F09325050E94A51A71F400E0FD
:101AFA0010E00C30E0E01E073CF40E94B71C0E9484
:101B0A001D1D0F5F1F4FF5CF35C0E130A0E0FA076A
:101B1A0071F400E010E00C30E0E01E073CF40E9493
:101B2A00CA1C0E941D1D0F5F1F4FF5CF23C0E23054
:101B3A00A0E0FA0771F400E010E00C30E0E01E07C4
:101B4A003CF40E94D51C0E941D1D0F5F1F4FF5CF4C
:101B5A0011C0E330A0E0FA0769F400E010E00C30AD
:101B6A00E0E01E073CF40E94E01C0E941D1D0F5F6E
:101B7A001F4FF5CF099119910895E8810E94A91A7A
:101B8A00E1F49B9B04C00E942D1D0E94321DCF9B35
:101B9A0004C00E942D1D0E943B1D0E94441D10F08E
:101BAA000E944C1D0E94711C0E944F1D0E94861C9F
:101BBA000E94541D0E94AE177EC1E130A0E0FA07D0
:101BCA00E1F49B9B04C00E945F1D0E94321DCF9BC3
:101BDA0004C00E945F1D0E943B1D0E94641D10F0FC
:101BEA000E94691D0E94711C0E944F1D0E946C1D5B
:101BFA000E94541D0E94AE175EC1E230A0E0FA07AF
:101C0A00E1F49B9B04C00E946E1D0E94321DCF9B73
:101C1A0004C00E946E1D0E943B1D0E94731D20F08D
:101C2A00E0E0F0E00E94F01C0E94711C0E947B1D03
:101C3A000E94541D0E94AE173EC1E330A0E0FA078D
:101C4A0029F59B9B04C00E94811D0E94321DCF9BD7
:101C5A0004C00E94811D0E943B1D0E94861D94970C
:101C6A0010F00E948B1D0E94861D1F9710F40E947F
:101C7A008B1D0E94711C0E948E1D0E94B41B0E9423
:101C8A00761C0E94541D0E94AE1715C1E430A0E0D4
:101C9A00FA0729F59B9B04C00E94931D0E94321DDE
:101CAA00CF9B04C00E94931D0E943B1D0E94981D59
:101CBA00949710F00E949D1D0E94981D1F9710F482
:101CCA000E949D1D0E94711C0E948E1D0E94131D60
:101CDA000E94761C0E94541D0E94AE17ECC0E5308B
:101CEA00A0E0FA07C9F49B9902C00E94A01DCF99EF
:101CFA0004C00E94E41A0E94A91D0E94A41B21F498
:101D0A000E946B1C0E94AF1D0E94891B21F40E9435
:101D1A006B1C0E94B21DCFC0E630A0E0FA0701F5A5
:101D2A009B9904C00E94F01A0E94A91DCF9908C06D
:101D3A00E0E0F0E0E0932805F09329050E94A91D50
:101D4A000E94181D309721F40E946B1C0E94AF1D3F
:101D5A000E94371C21F40E946B1C0E94B21DABC06A
:101D6A00E730A0E0FA0771F50E94181D309711F5C7
:101D7A009B9B04C00E94B51D0E94321DCF9B04C0CC
:101D8A000E94B51D0E943B1D0E943D1CAB3FE0E036
:101D9A00BE0720F0E0E0F0E00E94041D0E94711CE2
:101DAA00E5E4F3E00E94BA1D0E94BE1D0E94711C68
:101DBA000E94AE170E94371C21F40E946B1C0E94DD
:101DCA00B21D79C0E830A0E0FA0791F50E94181D0B
:101DDA00309731F59B9B04C0ACE2B5E00E94C31D6D
:101DEA00CF9B04C0ACE2B5E00E94C61DA0912C05B1
:101DFA00B0912D05AB3FE0E0BE0730F0E0E0F0E047
:101E0A00E0932C05F0932D050E94711C0E944F1D32
:101E1A000E94421C0E94761C0E94541D0E94AE170A
:101E2A000E94371C21F40E946B1C0E94B21D43C001
:101E3A00E930A0E0FA07D1F49B9B02C00E94C91DB9
:101E4A00CF9B02C00E94CC1D0E94CF1D10F00E94A1
:101E5A00D71D0E94711C0E94DA1D0E94DF1D0E947C
:101E6A00BE1D0E94711C0E94AE1725C0EA30A0E078
:101E7A00FA0709F59B9B04C0AAE3B5E00E94C31DBB
:101E8A00CF9B04C0AAE3B5E00E94C61D0E94CF1DE5
:101E9A0020F0E0E0F0E00E94091D0E94711C0E94FF
:101EAA00DA1D0E942B1B0E94761C0E94BE1D0E94F6
:101EBA00711C0E94AE1721960895E8810E94A91A02
:101ECA00E1F49B9B04C00E942D1D0E94321DCF9BF2
:101EDA0004C00E942D1D0E943B1D0E94441D10F04B
:101EEA000E944C1D0E94711C0E944F1D0E94861C5C
:101EFA000E94541D0E94AE1763C0E130A0E0FA07A9
:101F0A0029F59B9B04C00E94811D0E94321DCF9B14
:101F1A0004C00E94811D0E943B1D0E94861D949749
:101F2A0010F00E948B1D0E94861D1F9710F40E94BC
:101F3A008B1D0E94711C0E948E1D0E94B41B0E9460
:101F4A00761C0E94541D0E94AE173AC0E230A0E0EF
:101F5A00FA07C9F49B9902C00E94A01DCF9904C038
:101F6A000E94E41A0E94A91D0E94A41B21F40E9447
:101F7A006B1C0E94AF1D0E94891B21F40E946B1CDE
:101F8A000E94B21D1DC0E330A0E0FA07C9F49B9B72
:101F9A0002C00E94C91DCF9B02C00E94CC1D0E9494
:101FAA00CF1D10F00E94D71D0E94711C0E94DA1DDD
:101FBA000E94DF1D0E94BE1D0E94711C0E94AE1766
:101FCA0025C3E8810E94A91AE1F49B9B04C00E94E0
:101FDA005F1D0E94321DCF9B04C00E945F1D0E949C
:101FEA003B1D0E94641D10F00E94691D0E94711C15
:101FFA000E944F1D0E946C1D0E94541D0E94AE1724
:10200A008BC0E130A0E0FA07E1F49B9B04C00E9478
:10201A006E1D0E94321DCF9B04C00E946E1D0E943D
:10202A003B1D0E94731D20F0E0E0F0E00E94F01CCE
:10203A000E94711C0E947B1D0E94541D0E94AE17B3
:10204A006BC0E230A0E0FA0729F59B9B04C00E940E
:10205A00931D0E94321DCF9B04C00E94931D0E94B3
:10206A003B1D0E94981D949710F00E949D1D0E948E
:10207A00981D1F9710F40E949D1D0E94711C0E94BA
:10208A008E1D0E94131D0E94761C0E94541D0E94E0
:10209A00AE1742C0E330A0E0FA07C9F49B9902C028
:1020AA000E94A01DCF9904C00E94E41A0E94A91D93
:1020BA000E94A41B21F40E946B1C0E94AF1D0E9467
:1020CA00891B21F40E946B1C0E94B21D25C0E430BA
:1020DA00A0E0FA0709F59B9B04C0AAE3B5E00E94B9
:1020EA00C31DCF9B04C0AAE3B5E00E94C61D0E948F
:1020FA00CF1D20F0E0E0F0E00E94091D0E94711C53
:10210A000E94DA1D0E942B1B0E94761C0E94BE1D93
:10211A000E94711C0E94AE1779C20E94E11DA09113
:10212A005E05A33011F00C945D110E945C1C0E94A4
:10213A00E51D999B02C00E94E81D999902C0A895C5
:10214A00FCCF0E94EE1D9A9B02C00E94F41D9A9930
:10215A0002C0A895FCCF0E94EE1DA0915F05AB308E
:10216A0018F0E0E0E0935F050E94FA1D59F40E941E
:10217A00931C0E94FD1D0E949E1CE5E9F3E00E944B
:10218A00611C8DC0E130A0E0FA0749F40E94931C5B
:10219A000E94FD1D0E949E1C0E94001E80C0E2300B
:1021AA00A0E0FA0759F40E94931CEEEBF3E00E94B8
:1021BA00611C0E949E1C0E94031E71C0E330A0E0B5
:1021CA00FA0749F40E94931C0E94061E0E949E1C54
:1021DA000E94031E64C0E430A0E0FA0749F40E949A
:1021EA00931C0E94061E0E949E1C0E94091E57C034
:1021FA00E530A0E0FA0749F40E94931C0E940C1EE5
:10220A000E949E1C0E94001E4AC0E630A0E0FA0707
:10221A0059F40E94931CE7E2F4E00E94611C0E94B8
:10222A009E1C0E94001E3BC0E730A0E0FA0769F43A
:10223A000E94931CEEEBF3E00E94611C0E949E1C1C
:10224A00ECE3F4E00E94611C2AC0E830A0E0FA073F
:10225A0059F40E94931CE1E5F4E00E94611C0E947B
:10226A009E1C0E94001E1BC0E930A0E0FA0759F428
:10227A000E94931CE6E6F4E00E94611C0E949E1CE8
:10228A000E94031E0CC0EA30A0E0FA0741F40E9443
:10229A00931C0E940F1E0E949E1C0E94091EE09120
:1022AA005F05EA936ADC989902C00E94121E37CF32
:1022BA0008950E94E11DA0915E05A33011F00C94CF
:1022CA00C6110E945C1C0E94E51D999B02C00E94D7
:1022DA00E81D999902C0A895FCCF0E94EE1D9A9B11
:1022EA0002C00E94F41D9A9902C0A895FCCF0E94D0
:1022FA00EE1DA0915F05A43018F0E0E0E0935F05C1
:10230A000E94FA1D59F40E94931C0E94FD1D0E940E
:10231A009E1CE5E9F3E00E94611C2AC0E130A0E0BE
:10232A00FA0749F40E94931C0E94061E0E949E1CF2
:10233A000E94031E1DC0E230A0E0FA0759F40E9471
:10234A00931C0E940C1E0E949E1CEFE8F4E00E945F
:10235A00611C0EC0E330A0E0FA0751F40E94931CFE
:10236A00E6E6F4E00E94611C0E949E1C0E94031E85
:10237A00E0915F05EA93A1DD989902C00E94121EBE
:10238A009ACF08950E94E11DA0915E05A33011F035
:10239A000C943A120E945C1C0E94E51D999B02C093
:1023AA000E94E81D999902C0A895FCCF0E94EE1DD3
:1023BA009A9B02C00E94F41D9A9902C0A895FCCF6C
:1023CA000E94EE1DA0915F05A53018F0E0E0E093B1
:1023DA005F050E94FA1D49F40E94931C0E94FD1D8C
:1023EA000E949E1C0E94001E37C0E130A0E0FA073E
:1023FA0059F40E94931C0E94FD1D0E949E1CE4EA4F
:10240A00F4E00E94611C28C0E230A0E0FA0749F417
:10241A000E94931C0E94061E0E949E1C0E94091E76
:10242A001BC0E330A0E0FA0759F40E94931C0E94F3
:10243A000C1E0E949E1CE4EAF4E00E94611C0CC07F
:10244A00E430A0E0FA0741F40E94931C0E940F1E98
:10245A000E949E1C0E94091EE0915F05EA93B1DD6D
:10246A00989902C00E94121E8FCF0895E8810E9497
:10247A00A91AA1F59B9B04C0A2E4B5E00E94C31D62
:10248A00CF9B04C0A2E4B5E00E94C61DA0914205FC
:10249A00B0914305139710F00E94E41A0E94A41BFE
:1024AA0039F40E946B1CE9EBF4E00E94611C15C030
:1024BA00E130A0E0FA0739F40E946B1CEEECF4E07C
:1024CA000E94611C0AC0E230A0E0FA0731F40E94BF
:1024DA006B1CE3EEF4E00E94611C98C0E130A0E0BE
:1024EA00FA0741F50E94471CD8F49B9B04C00E943E
:1024FA005F1D0E94321DCF9B04C00E945F1D0E9477
:10250A003B1D0E94641D10F00E94691D0E94711CEF
:10251A000E944F1D0E946C1D0E94541D0E94AE17FE
:10252A000E94471C31F40E946B1CE8EFF4E00E9401
:10253A00611C6CC0E230A0E0FA0711F00C94E712BB
:10254A000E94A41BC9F49B9B02C00E94C91DCF9B79
:10255A0002C00E94CC1D0E94CF1D10F00E94D71D00
:10256A000E94711C0E94DA1D0E94DF1D0E94BE1D7E
:10257A000E94711C0E94AE170E94891B31F40E94AE
:10258A006B1CE8EFF4E00E94611C0E94471CC9F42E
:10259A009B9B02C00E94C91DCF9B02C00E94CC1DFA
:1025AA000E94CF1D10F00E94D71D0E94711C0E942C
:1025BA00DA1D0E94DF1D0E94BE1D0E94711C0E942E
:1025CA00AE1724C0E330A0E0FA0701F59B9B04C0D4
:1025DA000E94B51D0E94321DCF9B04C00E94B51DEA
:1025EA000E943B1D0E943D1CA53FE1E0BE0720F072
:1025FA00E0E0F0E00E94041D0E94711CEDE0F5E0AD
:10260A000E94BA1D0E94541D0E94AE172196089579
:10261A000E94E11DA0915E05A33011F00C9479137C
:10262A000E945C1C0E94E51D999B02C00E94E81D45
:10263A00999902C0A895FCCF0E94EE1D9A9B02C0F0
:10264A000E94F41D9A9902C0A895FCCF0E94EE1D23
:10265A00A0915F05A43018F0E0E0E0935F050E94C6
:10266A00FA1D69F40E94931CEBE1F5E00E94611CDB
:10267A000E949E1CE0E3F5E00E94611C2CC0E13040
:10268A00A0E0FA0749F40E94931C0E94FD1D0E94D3
:10269A009E1C0E94091E1FC0E230A0E0FA0759F4EE
:1026AA000E94931C0E940F1E0E949E1CE5E4F5E006
:1026BA000E94611C10C0E330A0E0FA0761F40E9496
:1026CA00931CEAE5F5E00E94611C0E949E1CE0E36F
:1026DA00F5E00E94611CE0915F05EA93C7DE9899D4
:1026EA0002C00E94121E96CF0895E0913E05F09115
:1026FA003F050E94571C999B11C00E94301B1B97D3
:10270A003CF00E94861A3A970E94211B0E94A91D3A
:10271A000E94301B1A9714F40E945A1B9A9B07C0F6
:10272A000E94861A3A960E94211B0E94A91D0E94A5
:10273A005D1B14F00E943C1B9B9B0EC00E94ED1B6C
:10274A001B9724F00E94241C0E94A91D0E94ED1BC5
:10275A001A9714F40E94CF1BCF9B09C00E94941AA7
:10276A003A96E0934805F09349050E94A91D0E94F4
:10277A00ED1BA536E0E0BE0714F00E94121C089576
:10278A000E94A51A19F40E94170721C0E130A0E09F
:10279A00FA0719F40E942B081AC0E230A0E0FA07DF
:1027AA0019F40E94B70813C0E330A0E0FA0719F43D
:1027BA000E9433090CC0E430A0E0FA0711F495DF57
:1027CA0006C0E530A0E0FA0711F40E94CA0908958C
:1027DA00A0915C05A33011F00C943E150E945C1C7C
:1027EA00EFE6F5E00E94611C0E946B1CE4E8F5E04C
:1027FA000E94611C99996A94999902C0A895FCCF84
:10280A000E94EE1D9A9963949A9902C0A895FCCFEA
:10281A000E94EE1DE6E0E61508F46624662089F4B7
:10282A000E94931CE9E9F5E00E94611C0E949E1C2B
:10283A00EEEAF5E00E94611C989903C0E1E0E0939A
:10284A005C05E1E0E61551F50E949E1CE3ECF5E01B
:10285A000E94611C0E94711CE8EDF5E0FA93EA936C
:10286A000E94191E0E94761C0E941E1E0E94711C44
:10287A000E94AE179B9B04C00E94191E0E94231E31
:10288A00CF9B04C00E94191E0E942D1E0E94191E71
:10289A00F39720F0A1EAB1E00E94DA1AE2E0E61525
:1028AA0051F50E949E1CE9EEF5E00E94611C0E940F
:1028BA00711CEEEFF5E0FA93EA930E94371E0E942C
:1028CA00761C0E941E1E0E94711C0E94AE179B9BC2
:1028DA0004C00E94371E0E94231ECF9B04C00E9480
:1028EA00371E0E942D1E0E94191EF39720F0A3EA9C
:1028FA00B1E00E94DA1AE3E0E61551F50E949E1C47
:10290A00EFE0F6E00E94611C0E94711CE4E2F6E02E
:10291A00FA93EA930E942B1C0E94761C0E941E1EA8
:10292A000E94711C0E94AE179B9B04C00E942B1C24
:10293A000E94231ECF9B04C00E942B1C0E942D1EA6
:10294A000E942B1CFD9720F0A7EAB1E00E94DA1A38
:10295A00E4E0E61509F50E949E1CE9E3F6E00E9410
:10296A00611CA0915D05A43029F40E94931CEEE439
:10297A00F6E004C00E94931CE4E6F6E0FA93EA93B8
:10298A000E94BB17989908C00E94931CEEE4F6E0D7
:10299A000E94611C0E94A305E5E0E615A9F50E94C4
:1029AA009E1CEAE7F6E00E94611C9B9905C0A5EA15
:1029BA00B1E0E0E00E946C1F9B9902C0A895FCCF91
:1029CA000E94EE1DCF9905C0A5EAB1E0E1E00E94A0
:1029DA006C1FCF9902C0A895FCCF0E94EE1D0E94E1
:1029EA00701A31F40E94931CEFE8F6E00E94611C11
:1029FA00A5EAB1E00E94581FE13031F40E94931C0D
:102A0A00E4EAF6E00E94611CE6E0E61589F50E9418
:102A1A009E1CE9EBF6E00E94611C0E943C1EE0301D
:102A2A0031F40E94931CEEECF6E00E94611C0E94B5
:102A3A003C1EE13031F40E94931CE3EEF6E00E9462
:102A4A00611C9B9905C0A6EAB1E0E1E00E94411E23
:102A5A00CF9905C0A6EAB1E0E0E00E94411E0E94BB
:102A6A003C1EE23028F0A6EAB1E0E0E00E946C1FCA
:102A7A00AFCE0E946F170E94651A08950E94491EE0
:102A8A001A930A931BB10CB1A12FB0E0ECE1F0E06C
:102A9A00EA23FB233097E1F4E091C405F0E0EE5617
:102AAA00FA4F0083A091C405AF5FA093C405A23377
:102ABA0019F4E0E0E093C405A091C605AF5FA093C6
:102ACA00C605A23329F4E0E0E093C605689420F82D
:102ADA000E94701A19F405D0E093400509911991E2
:102AEA0096C01A93E091C605E030E1F3E091C5057E
:102AFA00F0E0EE56FA4F1081A091C505AF5FA093A2
:102B0A00C505A23319F4E0E0E093C505F894E09115
:102B1A00C605E150E093C6057894E12F199108950E
:102B2A000E94491E552031F4E1E0E0935A05E0E0A5
:102B3A00E0935B05E1E0E51541F40E94C306E0E09D
:102B4A00E0935A05E2E0E0935B050E94A91D5FC08D
:102B5A000E94491E552041F5A0915905A73021F53B
:102B6A00442029F4E3E0E0935E050E949210E1E03C
:102B7A00E41529F4E3E0E0935E050E945E11E2E0C9
:102B8A00E41529F4E3E0E0935E050E94C711E3E04F
:102B9A00E41519F4E0935E053BDDE6E0E41521F463
:102BAA00E3E0E0935C0514DE32C00E94491EA6E30E
:102BBA00B5E00E94571E0E942E04E0915005E030B5
:102BCA0011F40E94FE1AA0915005A13021F4A3E548
:102BDA00B5E00E94571EE0915105E03011F40E94C1
:102BEA00051BA0915105A13021F4A5E5B5E00E948D
:102BFA00571EE0915205E03011F40E940C1BA0917F
:102C0A005205A13021F4A7E5B5E00E94571EE991CB
:102C1A00EFBFF991E991B991A99199918991799126
:102C2A006991F990199009901895E0E8EBBBEABB15
:102C3A00E0E0E8BBEFEFE7BBEFE6E5BBE0E9E4BBCA
:102C4A00E0E0E2BBE1BBE0E5E3B9E8E0E2B9E0E0FD
:102C5A00E0936200E0936100E0936500E093640012
:102C6A00E0BFE7E6E3BFE0E0E2BFE1BFE8EAEFBDCD
:102C7A00ECE0EEBDE0E0EDBDECBDE7BDE6BDEAE7A8
:102C8A00EBBDE2E1EABDE0E0E9BDE8BDE093790031
:102C9A00E0937800E0E1E7BFEBE6E5BDE0E0E4BD04
:102CAA00E3BDE1E8E0938B00E5E0E0938A00E0E031
:102CBA00E0938900E0938800E0938100E09380002C
:102CCA00E0938700E0938600E0938500E093840018
:102CDA00E0938300E0938200E0936A00EABFE0E5B4
:102CEA00E9BFE8BFE0E1E7BFE0E0E0937D00EBB9D0
:102CFA00E8E9EAB9E6E0E0939500E0E0E0939000C5
:102D0A00EFE2E9B9E0E8E8B9E0E0E0BDE3E5EDB912
:102D1A00E0E0EEB9E4E1EA930E94DD17EEE1E1BDFD
:102D2A00EEE0E1BD78940E946F170E94F71A4424DE
:102D3A00E1E0E0934005E0E0E09341055524E093AB
:102D4A006005BB24AA24DD24E7E0E0935905E0E00E
:102D5A00E0935A05E7E0E0935B05A8950E94651A9F
:102D6A004A920E94500A5A920E94160B0E94A01A76
:102D7A000E94761AFA93EA93E0914A05EA93E0915F
:102D8A004805EA930E942A0B0E94680B0E94740B62
:102D9A00552021F40E94960B0E94D20BE1E0E51522
:102DAA0021F44A920E94030AEBDC0E94941AEE0F65
:102DBA00FF1FE1BF0E94861AEE0FFF1FE0938600F5
:102DCA00A895442031F5E1E0E51589F4E4E04E16D2
:102DDA0070F49A9B05C00E945D1E3196FE93EE9395
:102DEA00999B05C00E945D1E3197FE93EE93A091B8
:102DFA004405B0914505A233E1E0BE0750F0AC327C
:102E0A00E1E0BE0720F4ECE2F1E00E94571C0E94C8
:102E1A004C1D552019F49A9901C0FDCF0E94550402
:102E2A00A8959BCFFFCFFFE0FA95F1F70895A1B3DC
:102E3A00AF70A1BB919A9098F6DF929AF4DFA0B393
:102E4A009298F1DF929AEFDF9298A7FDF5CF089555
:102E5A00A07FAB2BA2BB929A0E94181792980E944D
:102E6A00181708959198A1B3A76FA1BBB2B3BF7009
:102E7A00A881EEDFA881A295EBDF919A0C94251A1E
:102E8A00929A0E941817E0B392980E941817E07F4E
:102E9A0008950E941817F4DFAE2FF2DF9198E29599
:102EAA00EA2B08950E941C170E94641EE953FA4FE8
:102EBA00E081F0E0DF01E981F0E0EA0FFB1FEA932D
:102ECA000E943717E981E093CB05E881E093CC05AE
:102EDA00229608950E941C17E2E0EA930E9437178F
:102EEA000E941C17ECE0EA930E9437170E941C17F5
:102EFA00E1E0EA930E943717E0E0E093CC05E09323
:102F0A00CB050895EF93FF93A8816894AA3061F0E6
:102F1A00E894E091CB05EF5FE093CB05E091CD0516
:102F2A00A091CB05EA1760F4E091CC05EF5FE0933E
:102F3A00CC05E0E0EA93E091CC05EA93B3DF2EF00A
:102F4A0076DF909AA881AA938DDFFF91EF910C9476
:102F5A00251A1A93A981BA81ED91A983BA831E2FE2
:102F6A00E03019F01A93CEDFF5CF0EC01A93E9813B
:102F7A00FA813196E983FA833197E4911E2FE03082
:102F8A0019F01A93BFDFF3CF188123960895AA2761
:102F9A00BB271197F1F708959198A1B3A76FA1BB29
:102FAA00B2B3BF70A8810E942D17919A0C94251A6A
:102FBA0092989098E881E093CD050E94641EE058AB
:102FCA00FF4FE093C9050E94641EE054FF4FE0934F
:102FDA00CA050E94671E0E94671E0E94671ED7DFED
:102FEA00E0E2EA93D9DFD3DFEAE20E946D1EE4E071
:102FFA000E946D1EE5E80E946D1EA1B3AF70A1BBD1
:10300A00919A0E944E17E53019F0E0E00C94251AC7
:10301A000E941C17E6E0EA930E9437170E946F1776
:10302A00E1E00C94251A5D9BFECFE881ECB908C259
:10303A001A930A93AC81BD810E94351F3097C1F063
:10304A00AA81BB810E94351F8F01309749F0023057
:10305A00E0E01E0760F0F80131978F01ED93FC93D1
:10306A00AC81BD810E94571E3197AE81A08303C0F7
:10307A00EE81EA93D8DF1981088127960895269769
:10308A000E94F72010E0EA89FB893196EA8BFB8BD4
:10309A003197E4912E2FE03011F40C94F519E12FB9
:1030AA000E94A91A39F4253211F411E002C00E94D3
:1030BA00721E95C1E130A0E0FA07A9F4253219F48D
:1030CA000E94721E8BC112E040E000E02D3211F422
:1030DA0001E085C12B3211F44BE281C1203211F497
:1030EA0040E27DC104C0E230A0E0FA0761F450E09A
:1030FA0013E0203339F40E947D1EE0E8F0E0EA2B69
:10310A000E2F6DC106C0E330A0E0FA0711F00C944F
:10311A00F419203310F02A3308F015C0A52FB0E0B7
:10312A00EAE0F0E0EA02F0015E2F652F7727A22F8E
:10313A00B0E0E0E3F0E00E944D1FEA1BFB0BDB016D
:10314A00EA0F5E2F4CC10E94801EE336A0E0FA0708
:10315A0049F40E94831EE889F989A481AA930E94EE
:10316A00891E3CC1E337A0E0FA0741F40E94831E9E
:10317A000E94931E0E94271A1E2F11C0E037A0E05A
:10318A00FA07D9F40E94831E0E94931E0E94311AE4
:10319A001E2F0E947D1EE8E0F0E0EA2B0E2F0E940F
:1031AA007D1EE2E0F0E0EA2B0E2F0E947D1EEFE783
:1031BA00FFEFEA230E2F30E04FC0E436A0E0FA0713
:1031CA0021F0E936A0E0FA0739F40E947D1EE4E016
:1031DA00F0E0EA2B0E2F04C0E537A0E0FA0731F43D
:1031EA00ECE8F0E0EE83FF8315E016C0E835A0E0D6
:1031FA00FA0739F40E947D1EE8E0F0E0EA2B0E2F70
:10320A0006C0E837A0E0FA0711F00C94F319E6E9D2
:10321A00F0E0EE83FF8314E00E947D1E0E949D1E53
:10322A00B9F00E94831E0E94A31EAB85AA233AF41A
:10323A00EA85FB850E94E51EEA87FB874DE240305E
:10324A0011F01F5F04C00E947D1E0E94AB1E04C0C5
:10325A000E94831E0E94A31E0E94B01EE9F4151745
:10326A00D8F40E947D1EE0E8F0E0EA23FB233097C1
:10327A0071F00E947D1E0E949D1E39F00E947D1EE3
:10328A000E94AB1E242F115001C020E301C020E28E
:10329A000E94721E5150E3CF312F0E947D1EE2E040
:1032AA00F0E0EA23FB23309701F13030E9F00E9485
:1032BA007D1EE8E0F0E0EA23FB23309741F0EE813F
:1032CA00FF813196EE83FF833197E49105C0AE8189
:1032DA00BF81ED91AE83BF83EA930E94891E50306D
:1032EA0009F051503150E1CF6EC020E3EE81FF81E9
:1032FA000E94391FE887F987EE81FF813296EE83B3
:10330A00FF83E885F985AA85BB85AE17BF0750F00C
:10331A002F5FA885B985EA85FB85EA1BFB0BEA873F
:10332A00FB87EFCF2A3380F00E947D1EE8E0F0E0B1
:10333A00EA23FB23309721F00E94801E379603C0B0
:10334A000E94801EB7962E2F0E947D1EE0E1F0E0BB
:10335A00EA23FB23309761F5213320F4A885B98548
:10336A00119709F410C0531718F00E94B01E09F003
:10337A0024C020E20E947D1EE0E8F0E0EA23FB235D
:10338A003097B1F020E3A02FB0E0E0E1F0E0EA2BC3
:10339A000E2F0E947D1E0E949D1E51F00E947D1ECE
:1033AA000E94AB1E4A930E94891E503009F0515068
:1033BA000E94721E503009F051503150A885B985CB
:1033CA00129708F092CF0E94B01E41F0503031F0AF
:1033DA005150E0E2EA930E94891EF8CF10E053CEE2
:1033EA000E94FE2064960895FF920E94B41EDE0198
:1033FA0016960E94BD1EEA83FB83DE0114960E9484
:10340A00BD1E0E94C21EAA81BB81E0E0EC930CC0E3
:10341A00FF920E94B41EE0E0EA83EB83DE01149679
:10342A000E94BD1E0E94C21E198108812496FF9027
:10343A000895E881EFB9EEB1F0E0E078E1F3EFB199
:10344A0021960895A991B991EE27FF276D916623D8
:10345A0011F03196FBCF0895AA27BB27E991F9917C
:10346A000590002011F01196FBCFFD010895E3E5C8
:10347A00EDB9E0E0EEB9B99ABA9ABB980895E0E0DE
:10348A00EA930E941E1AF0E0089566277727DF0163
:10349A00CB01E8E00E94F11E0895662777270E9473
:1034AA00E01E8F01087F1F771695079516950795D9
:1034BA00169507950895A0913C05B0913D0508958C
:1034CA00E8ECF0E0FA93EA930C94D01EA0913E0542
:1034DA00B0913F050895A5EAB1E00E94581FE03077
:1034EA000895FA93EA93E0913E05F0913F05089515
:1034FA00662777270E943D1F84E00E940D1A2696B0
:10350A000895E0914A05F0914B0508950E94FD1E29
:10351A000E943D1F84E00E940D1A26960895E091AC
:10352A004805F09149050895FA93EA9380E00E94CC
:10353A000D1A22960895E0913C05F0913D050895F3
:10354A00E42DF0E030970895F0E030970895EBE32A
:10355A00F1E0EACFE9E4F1E0E7CFE2E5F1E0E4CF38
:10356A00ECE2F1E0FA93EA930C94D01EE0E0F0E08A
:10357A00E0934405F0934505E0934605F09347052B
:10358A00E0934A05F0934B05E0934805F09349050B
:10359A00882499240895E4EFF1E00E94641F0895B5
:1035AA00E6E1F0E00E94641F0895E0E0F0E00E9486
:1035BA00641F0895E4E6F0E00E94641F0895E0E0C5
:1035CA00F0E0E0934205F09343050895E0932E0559
:1035DA00F0932F050895E1E0F0E0E0932805F093D9
:1035EA0029050895E0E0F0E0E0933605F093370509
:1035FA000895E0E0F0E0E0935305F0935405089550
:10360A00E0E0F0E0E0935505F09356050895E0E018
:10361A00F0E0E0935705F09358050895E09191057D
:10362A00ADE6B5E0F0E0EE0FFF1FAE0FBF1F089545
:10363A00E0919105F0E00895E0934A05F0934B0577
:10364A000895A0914605B09147050895E0913A057D
:10365A00F0913B050895A0914A05B0914B05089554
:10366A00F5DFEACF28DFAC32E1E0BE070895E4E6F1
:10367A00F0E0E2CF20DFAD32E1E0BE070895EAE0F4
:10368A00F0E0DACFE0913205F0913305A0913605EA
:10369A00B09137050E94071FDF01EAE0F0E00E94BF
:1036AA00141F94DFD8DF11970895E0E0F0E0C4CF4B
:1036BA00D2DFA536E0E0BE070895E0914605F09115
:1036CA004705A0912E05B0912F050895E0912E058A
:1036DA00F0912F05F0DEAE17BF070895AAE4B5E012
:1036EA00ED91FD9108953196FE93EE93AFDFB3DF2E
:1036FA00EA17FB070895E0914C05F0914D050895EE
:10370A00E5DEEA17FB070895A0914205B09143054B
:10371A0011970895F0DFDADEAE17BF0708950BDFC1
:10372A00EA55F040E0936305F09364050895E0914B
:10373A006305F0916405FA93EA930C94D506E09137
:10374A004205F091430530970895E0914605F091BE
:10375A004705EA55F040FA93EA930C94D506E091AE
:10376A003405F09135050895A0915305B09154059B
:10377A0008950E94071FDF01EAE0F0E00E94141F8B
:10378A00E0934E05F0934F05A0914805B091490585
:10379A0011970895E0E0F0E0E0934805F0934905B9
:1037AA000895E0914405F09145050895A0914E05CC
:1037BA00B0914F05EA17FB070895F3DFE0934E0532
:1037CA00F0934F050895E0913805F0913905089571
:1037DA00A0914805B09149050895F5DFE0934805A1
:1037EA00F09349050895DDDF71DEAE17BF0708952E
:1037FA00E0914E05F0914F0569DEAE17BF070895B7
:10380A00A8E4B5E0ED91FD9108953196FE93EE930B
:10381A00DFDFA536E0E0BE070895E4E6F0E0E093D6
:10382A004805F09349050895A0914405B0914505CE
:10383A00E0913E05F0913F05EA1BFB0B08956FDE10
:10384A003A97E0934805F09349050895A7EAB1E04D
:10385A000E94541F0895A0915705B0915805EA1780
:10386A00FB070895A0912805B0912905119708959D
:10387A00A0912A05B0912B050895E0912C05F091AD
:10388A002D050895A0914205B09143051297089518
:10389A00E0914605F09147050895E0912A05F091D7
:1038AA002B050895E0934405F09345050895E0E05B
:1038BA00EA93EA930C945717FA93EA930C94BB177A
:1038CA00EAE0EA93E0E0EA930C945717E0E0EA931F
:1038DA00E1E0EA930C945717E0E0F5E0FA93EA93F3
:1038EA000895662777270E943D1F08958CE00E945D
:1038FA00F9196096E0E0EA930895E2E0EA930C94FD
:10390A0057174FDFEECFE3E0EA930C945717B0E076
:10391A00E1E0F0E00E944D1FEA1B0895E0E0EA931F
:10392A00ECCFE5EAF2E0C8CFE0E0E09359054A922D
:10393A000895E0E0EA93E7CFEEE1F0E0FA93EA9344
:10394A000E94D01EB4CF0E94500AF3CFEFECF2E0EF
:10395A00B3CFF801A0E1B5E0EE0FFF1FEA0FFB1F9E
:10396A00BF010895E72DA8E1EA9FF001E050F04079
:10397A00DF01F801EE0FFF1F0895AE0FBF1F0E946F
:10398A00541FDB01ED93FC930895EA2DA8E1EA9F09
:10399A00F001E054FF4FDF01F801EE0FFF1F089519
:1039AA00EB2DA8E1EA9FF001E85FFE4FDF01F80185
:1039BA00EE0FFF1F0895ED2DA8E1EA9FF001E05BED
:1039CA00FE4FDF01F801EE0FFF1F0895E093460551
:1039DA00F09347050895E0934C05F0934D0508953B
:1039EA00E0933405F09335050895E0933205F0939A
:1039FA0033050895E0934205F09343050895E09353
:103A0A002A05F0932B050895E0933A05F0933B05B8
:103A1A000895E0933805F09339050895E091320549
:103A2A00F09133050895E0912805F091290508954C
:103A3A00EA0FFB1F0F01F801A0E1B5E0EE0FFF1F2F
:103A4A00AE0FBF1F0E94351FD0010E94641F089548
:103A5A00A4E4B5E0ED91FD9108953197FE93EE93BC
:103A6A00E2E3F0E0FA93EA930C94D01E3196FE93C7
:103A7A00EE93E2E3F0E0FA93EA930C94D01EA0915D
:103A8A004405B0914505AD32E1E0BE070895E0E096
:103A9A00F0E008CFE4EEF2E0FA93EA93089584E0C6
:103AAA000E94F9192896E2E0EA93E1E0EA930E947B
:103ABA00571712CFA6E4B5E0ED91FD910895C1DD47
:103ACA00A53FE1E0BE070895E0E0F0E07FCFE0DE49
:103ADA0008CFACE4B5E0ED91FD910895A0914C05B5
:103AEA00B0914D05AB3FE0E0BE070895E3EFF2E089
:103AFA00FA93EA9300DEF5CEA4E3B5E0ED91FD91E9
:103B0A000895A0913405B09135050895EFE0F0E0ED
:103B1A0067CFE7E0F3E0FA93EA930895A2E3B5E00A
:103B2A00ED91FD910895A0913205B0913305089564
:103B3A00EFE0F0E05ACFE1E0F0E05CDFE2E3F0E052
:103B4A00FA93EA930C94D01EE2E3F0E0FA93EA9334
:103B5A000C94D01EEBE1F3E0AFCEE0E3F3E0ACCEA1
:103B6A00AAE2B5E0ED91FD910895FA93EA9395DE04
:103B7A00B8CE84E00E94F9192896A8CEED91FD915D
:103B8A006CCFED91FD9172CFA8E3B5E0F7CFA8E332
:103B9A00B5E0F7CFA0913805B0913905A536E0E038
:103BAA00BE070895E0E0F0E034CFE7E5F3E0FA93EA
:103BBA00EA93089508DE95CE0E946F170C949A0C2A
:103BCA00EBE6F3E079CEE0915F05E150E0935F0523
:103BDA000895EEE1F0E0FA93EA930C94D01EE09196
:103BEA005F05EF5FE0935F050895E0915F05ACCC58
:103BFA00E0E8F3E061CEEAEAF3E05ECEE3EDF3E07B
:103C0A005BCEE8EEF3E058CEEDEFF3E055CEE2E11D
:103C1A00F4E052CEEBE7F4E04FCE0E94330DE1E040
:103C2A00E0935E050C946F17A1EAB1E00E94541F5D
:103C3A00089584E00E94F919289670CE31970E945F
:103C4A00641F3196E4E6F0E0FA93EA930C94D01EEE
:103C5A0031960E94641F3197E4E6F0E0FA93EA9302
:103C6A000C94D01EA3EAB1E00E94541F0895A6EA5C
:103C7A00B1E00E94581F08950E946C1FE4E6F0E02C
:103C8A00FA93EA930C94D01E0A921A92FA926A93C1
:103C9A007A938A939A93AA93BA93EA93FA93EFB789
:103CAA00EA930895ED91FD913196FE93EE9308956E
:103CBA00E9E1F0E0FA93EA930E94D01EC9CEE881C6
:103CCA00F0E008950E94CC17E0E3EA930C94D11730
:103CDA00EA930E9437170C94CC172A93EF85F88938
:103CEA00FA93EA93FE013F96FA93EA930C941D180D
:103CFA00A02FB0E00895E22FF0E00895E889F9894D
:103D0A003497E88BF98B0895EF85F889FA93EA934B
:103D1A00FE013F96FA93EA930C941D18A889B98973
:103D2A0014960E94351FEE83FF83FA93EA9308954F
:103D3A00E4E0F0E0EA23FB2330970895A889B989E3
:103D4A0014960E94351FEA87FB870895EBEFFFEF71
:103D5A00EA230E2F0895E02FF0E0E1700895F82E7F
:103D6A0022971A930A93DE010E94DC1E8D010895A0
:103D7A000E94DC1E0E94351F0895FA93EA931A9353
:103D8A000A93FE013696FA93EA93E0E0F0E0FA939A
:103D9A00EA930C944418E991F991309639F083E347
:103DAA0097E00197F1F7A8953197C9F7089500248C
:103DBA00AF0DB01D0895EA2BFB2B682B792B0895C4
:103DCA00F195E195F0400895F09560957095E1952B
:103DDA00FF4F6F4F7F4F0895EE230E2EFD01BC015A
:103DEA0031F0EE0FFF1F661F771F0A94D1F708956F
:103DFA006F2F660F660B762F08958B2F880F880B0F
:103E0A00982F0895FA9FF02DEB9FF00DEA9FE02D71
:103E1A00F10D089517D0F6DF0EF4D2DF08950024CD
:103E2A00112490E1AA0FBB1F001C111C0E1A1F0AB5
:103E3A0018F40E0E1F1E01C0A1609A9599F7FD0194
:103E4A00D0010895E894F7FF02C0BADF6894B7FF7B
:103E5A0006C0A095B095119600F8039400FA08954B
:103E6A00ED91FC91119708950590F491E02D089534
:103E7A007A936A93FA93EA930895689401C0E8944E
:103E8A0001D09DD0182E862F612D192E972F712DB6
:103E9A001B2EBF2FF12D1A2EAE2FE12D089511964C
:103EAA0002D0FE2F1197E199FECFFF93FFB7F89446
:103EBA00AEBBBFBBE09AEDB3FFBFFF91089507D039
:103ECA001196EF93EF2F03D0EF9111970895E19B8D
:103EDA0002C0A895FCCF9FB7F894AEBBBFBBE09ACF
:103EEA008DB3E81719F0EDBBE29AE19A9FBF0895E6
:103EFA00552342F4503811F4E0FF04C03196691F8B
:103F0A00791F6BF050E8572711F45F93C6C05F3FE3
:103F1A0031F0660F000C57956795752F08955F93DA
:103F2A0000200AF0C6C0BFC050E8192E1522880F1B
:103F3A00991F9527550F879550E8072E0522660F7A
:103F4A00771F7527550F67950895689401C0E894FF
:103F5A005F93F2DF703818F07F3F08F49EC056E195
:103F6A00571BAAF4519558300EF4593030F0EFEF40
:103F7A00FFEF6FEF7FE777F91AC077275523B9F07C
:103F8A00EE0FFF1F661F771F5A95D1F710C07727CC
:103F9A00583028F0EF2FF62F672F5850F9CF5523B6
:103FAA0031F076956795F795E7955A95D1F7002000
:103FBA000AF40ADF5F910895689401C0E894309783
:103FCA0060407040B1F0002426F0772312F4009488
:103FDA00FBDE172E7EE1112032F07A95EE0FFF1FDD
:103FEA00661F111CF9CFEF2FF62F612D5F938ADF21
:103FFA005F9108954F93AF01FD01DA01AB01BC0156
:10400A00CA01402D012C142E4F910895EA0FFB1F6F
:10401A00681F0895E095F0956095EF5FFF4F6F4F29
:10402A0008955F9381DF903839F1703821F1572F65
:10403A00591B13F112F4DEDFFACF583118F0AA2710
:10404A00BB278827583028F0AB2FB82F882758501D
:10405A00F9CF552329F08695B795A7955A95D9F79B
:10406A00502D512562F0D2DF38F46795F795E79520
:10407A00739513F41EC0BEDF45DF5F910895EA1BF6
:10408A00FB0B680B51F010F40094C4DF6623A2F313
:10409A00EE0FFF1F661F7A95CBF7EE27FF276627DD
:1040AA0077275F910895EFEFFFEF6FE77FEF5F915B
:1040BA000895EFEFFFEF6FE77FE75F9108955F9352
:1040CA0033DF703851F3903841F301240894791F93
:1040DA0023F41CF300203AF3ECCF0F921F932F9393
:1040EA003F934F93112722279927689FA0018F9FFB
:1040FA00302D410D591F6B9F300D411D591F8E9F49
:10410A0027D0BF9F25D06A9F23D0BE9F1DD0AF9FC7
:10411A001BD0AE9F110D291F391F491F591FE32FAD
:10412A00F42F652F522F4F913F912F911F910F908E
:10413A0066232AF0550FEE1FFF1F661F02C07395F4
:10414A004BF2D6DE5F910895100D211D391F02C072
:10415A00200D311D491F591F08955F93E5DE703800
:10416A0021F411200AF49FCFA4CF903809F495CFF7
:10417A0001240894970B1BF4D4F30020F3CF792F72
:10418A001F932F933F934F931124112722273327ED
:10419A004427552790E2AE17BF078607410730F03C
:1041AA00AE1BBF0B860B410B089401C08894551FA8
:1041BA00221F331F111CAA1FBB1F881F441F9A9559
:1041CA0051F7F901612D4F913F912F911F9166236C
:1041DA0032F0550FEE1FFF1F661F7A9543F288DEF5
:1041EA005F9108955A934A933A932A931A930A939A
:1041FA0008955D814C813B812A8119810881089546
:00000001FF
:00000001FF
